:100000000C947B030C9495210C94C2210C94A303B3
:100010000C94A3030C94A3030C94A3030C94A303C8
:100020000C94A3030C94A3030C94A3030C94A303B8
:100030000C94A3030C94A3030C94A3030C94A303A8
:100040000C94EF210C94A3030C94B2230C9404247D
:100050000C94A3030C94A3030C94A3030C94A30388
:100060000C94B01F0C94A3030000211042206330B5
:100070008440A550C660E770088129914AA16BB100
:100080008CC1ADD1CEE1EFF13112100273325222A8
:10009000B5529442F772D662399318837BB35AA350
:1000A000BDD39CC3FFF3DEE3622443342004011478
:1000B000E664C774A44485546AA54BB528850995A0
:1000C000EEE5CFF5ACC58DD5533672261116300648
:1000D000D776F6669556B4465BB77AA719973887F0
:1000E000DFF7FEE79DD7BCC7C448E5588668A77808
:1000F0004008611802282338CCC9EDD98EE9AFF940
:10010000488969990AA92BB9F55AD44AB77A966AE7
:10011000711A500A333A122AFDDBDCCBBFFB9EEB8F
:10012000799B588B3BBB1AABA66C877CE44CC55CB7
:10013000222C033C600C411CAEED8FFDECCDCDDDDF
:100140002AAD0BBD688D499D977EB66ED55EF44E87
:10015000133E322E511E700E9FFFBEEFDDDFFCCF2F
:100160001BBF3AAF599F788F8891A981CAB1EBA183
:100170000CD12DC14EF16FE18010A100C230E320FF
:100180000450254046706760B9839893FBA3DAB3A7
:100190003DC31CD37FE35EF3B1029012F322D2324F
:1001A0003542145277625672EAB5CBA5A895898577
:1001B0006EF54FE52CD50DC5E234C324A01481049F
:1001C0006674476424540544DBA7FAB79987B89747
:1001D0005FE77EF71DC73CD7D326F2369106B016EF
:1001E00057667676154634564CD96DC90EF92FE907
:1001F000C899E9898AB9ABA944586548067827683F
:10020000C018E1088238A3287DCB5CDB3FEB1EFBE6
:10021000F98BD89BBBAB9ABB754A545A376A167A8E
:10022000F10AD01AB32A923A2EFD0FED6CDD4DCDB6
:10023000AABD8BADE89DC98D267C076C645C454CDE
:10024000A23C832CE01CC10C1FEF3EFF5DCF7CDF86
:100250009BAFBABFD98FF89F176E367E554E745E2E
:10026000932EB23ED10EF01E000000000000005F91
:1002700000000007000700147F147F14242A7F2A3F
:100280001223130864623649562050000807030001
:10029000001C2241000041221C002A1C7F1C2A084D
:1002A000083E080800807030000808080808004070
:1002B00000000020100804023E5149453E00427FE4
:1002C000400072494949462141494D331814127F73
:1002D0001027454545393C4A494931412111090713
:1002E0003649494936464949291E00140000000094
:1002F0004034000000081422411414141414004166
:1003000022140802015909063E415D594E7C121122
:10031000127C7F494949363E414141227F4141415A
:100320003E7F494949417F090909013E41415173D5
:100330007F0808087F00417F41002040413F017F46
:10034000081422417F404040407F021C027F7F040E
:1003500008107F3E4141413E7F090909063E415157
:10036000215E7F09192946264949493203017F0147
:10037000033F4040403F1F2040201F3F4038403F48
:10038000631408146303047804036159494D43005E
:100390007F4141410204081020004141417F040295
:1003A000010204404040404000030708002054542C
:1003B00078407F284444383844444428384444280A
:1003C0007F385454541800087E090218A4A49C785D
:1003D0007F0804047800447D40002040403D007FB9
:1003E0001028440000417F40007C047804787C0899
:1003F0000404783844444438FC182424181824246D
:1004000018FC7C08040408485454542404043F4451
:10041000243C4040207C1C2040201C3C4030403C80
:1004200044281028444C9090907C4464544C4400E0
:100430000836410000007700000041360800020144
:1004400002040202050200000E1111110E7A048E40
:10045000040000000000000000000021007F2200D6
:1004600007AED580A83FD300408D142000A1C8DA84
:100470001281CFD9F1DB40A4A6AFA204B804C7040F
:10048000DC04F104010513052705340548055C0566
:1004900082059405BF05E105FB05150635064A06EC
:1004A0006E064AFCFE0783C3E3733FFEFC4A0F1F40
:1004B0003F33313030381F0F02420C0EC204024667
:1004C00030303F3F3030024A0C0E07030383C3E74E
:1004D0007E3C4730383C3E37333183304A0C0E0780
:1004E0000303C3C3C7FE3C430C1C38843043381F8E
:1004F0000F46C0E070381C0EC2028603443F3F0323
:1005000003823F85334373E3C3430C1C3884304379
:10051000381F0F43FCFEC784C343C78E0C430F1F15
:1005200038843043391F0F840346C3E3733B1F0FE6
:1005300004823F04433CFEE784C343E7FE3C430F91
:100540001F39843043391F0F433C7EE784C343E7A0
:10055000FEFC02823046381C0E07030144F8FCFE04
:100560000E85074687C7EEFEFCF8C348E070381CCE
:100570000E07030101C34403070F0E871C440E0F2F
:1005800007030343080C0EC30606C30603831C833C
:100590001F831C0344383C3E0E87074406FEFCF8CC
:1005A000034C80C0E0F0783C1E0F07030100421CA2
:1005B0001E831F411D891C1C1C1C1C1C1C1C1C4454
:1005C000383C3E0E87074406FEFCF8838004840E08
:1005D000443FFFF1E04403070F0E871C440E0F0752
:1005E00003024780C0E0F0783C1EC303457E7F7F56
:1005F00073718470C3837009831F03C388C78287A4
:100600008207838188014103C34403070F0E871CBF
:10061000440E0F070344F8FCFE0E8707440E3E3CD1
:1006200038C3880E441CFCF8F04403070F0E871CE7
:10063000440E0F070388074787C7E7F77F3F1F066A
:1006400041FEC282010406831F0644F8FCFE8E8729
:1006500007448EFEFCF844E0F1FB3F870E443FFB6D
:10066000F1E04403070F0E871C440E0F070344F804
:10067000FCFE8E8707448EFEFCF80182034107834F
:100680000E488ECEEEFEFF7F3F0702831C461E1FE4
:100690000F0703010400000000240027002A0000C7
:1006A000000000250028002B000000000023002689
:1006B00000290004040404040404040202020202E7
:1006C0000203030303030301020408102040800116
:1006D0000204081020010204081020000000070096
:1006E00002010000030406000000000000000000FA
:1006F0009A09A61E732511241FBECFEFD8E0DEBFD6
:10070000CDBF11E0A0E0B1E0E4E4F5E502C0059062
:100710000D92AA37B107D9F718E0AAE7B1E001C0F6
:100720001D92A133B107E1F716E0C6EFD6E004C091
:100730002297FE010E949C2AC03FD107C9F70E9460
:10074000CA250C94A02A0C94000061E070E040E0FF
:1007500050E016C0342F2227FB01E254FA4F80816B
:10076000E82FF0E0852F9927E827F927EE0FFF1FE4
:10077000E859FF4F45915491422753276F5F7F4FB0
:100780008091F6059091F705861797071CF740931F
:100790000E0650930F06E091F605F091F705E05430
:1007A000FA4F4083E091F605F091F705E154FA4FD6
:1007B00050838091F6059091F70502969093F70586
:1007C0008093F6050895AF92BF92CF92DF92EF9299
:1007D000FF920F931F93CF93DF93109253051092C4
:1007E00052058FEF809356051092550510925405CF
:1007F0008AEE80938C0186EA80938D0110928E019F
:1008000084E090E09093E3048093E20483E090E03E
:100810009093E5048093E40440E050E0C1E0D0E030
:1008200031E0E32EF12C012D112D1092550510927F
:100830005405BE01042E02C0660F771F0A94E2F72A
:1008400066C08091540590915505FC01EE0FFF1F85
:10085000E80FF91FE250FB4F808190E08623972339
:10086000892BB9F0E091E404F091E504E557FE4FDF
:1008700020818091E2049091E3045701680104C053
:10088000AA0CBB1CCC1CDD1C8A95D2F72A2920831C
:1008900019C0E091E404F091E504E557FE4F208192
:1008A0008091E2049091E3045701680104C0AA0C0E
:1008B000BB1CCC1CDD1C8A95D2F7D601C5018095E6
:1008C000822380838091E2049091E30401969093C7
:1008D000E3048093E2048091E2049091E30408979A
:1008E0006CF01092E3041092E2048091E404909181
:1008F000E50401969093E5048093E4048091540507
:1009000090915505019690935505809354058091DB
:100910005405909155054C970CF493CF4F5F5F4F62
:100920004830510509F081CF40E050E0C1E0D0E00F
:10093000B1E0EB2EF12C012D112D109255051092E6
:100940005405BE01042E02C0660F771F0A94E2F719
:1009500066C08091540590915505FC01EE0FFF1F74
:10096000E80FF91FE250FB4F818190E08623972327
:10097000892BB9F0E091E404F091E504E557FE4FCE
:1009800020818091E2049091E3045701680104C042
:10099000AA0CBB1CCC1CDD1C8A95D2F72A2920830B
:1009A00019C0E091E404F091E504E557FE4F208181
:1009B0008091E2049091E3045701680104C0AA0CFD
:1009C000BB1CCC1CDD1C8A95D2F7D601C5018095D5
:1009D000822380838091E2049091E30401969093B6
:1009E000E3048093E2048091E2049091E304089789
:1009F0006CF01092E3041092E2048091E404909170
:100A0000E50401969093E5048093E40480915405F5
:100A100090915505019690935505809354058091CA
:100A20005405909155054C970CF493CF4F5F5F4F51
:100A30004430510509F081CF44E050E0C1E0D0E0FE
:100A400031E0E32EF12C012D112D1092550510925D
:100A50005405BE01042E02C0660F771F0A94E2F708
:100A600066C08091540590915505FC01EE0FFF1F63
:100A7000E80FF91FE250FB4F818190E08623972316
:100A8000892BB9F0E091E404F091E504E557FE4FBD
:100A900020818091E2049091E3045701680104C031
:100AA000AA0CBB1CCC1CDD1C8A95D2F72A292083FA
:100AB00019C0E091E404F091E504E557FE4F208170
:100AC0008091E2049091E3045701680104C0AA0CEC
:100AD000BB1CCC1CDD1C8A95D2F7D601C5018095C4
:100AE000822380838091E2049091E30401969093A5
:100AF000E3048093E2048091E2049091E304089778
:100B00006CF01092E3041092E2048091E40490915E
:100B1000E50401969093E5048093E40480915405E4
:100B200090915505019690935505809354058091B9
:100B30005405909155054B970CF493CF4F5F5F4F41
:100B40004830510509F081CF40E050E0C1E0D0E0ED
:100B5000B1E0EB2EF12C012D112D109255051092C4
:100B60005405BE01042E02C0660F771F0A94E2F7F7
:100B700066C08091540590915505FC01EE0FFF1F52
:100B8000E80FF91FE250FB4F828190E08623972304
:100B9000892BB9F0E091E404F091E504E557FE4FAC
:100BA00020818091E2049091E3045701680104C020
:100BB000AA0CBB1CCC1CDD1C8A95D2F72A292083E9
:100BC00019C0E091E404F091E504E557FE4F20815F
:100BD0008091E2049091E3045701680104C0AA0CDB
:100BE000BB1CCC1CDD1C8A95D2F7D601C5018095B3
:100BF000822380838091E2049091E3040196909394
:100C0000E3048093E2048091E2049091E304089766
:100C10006CF01092E3041092E2048091E40490914D
:100C2000E50401969093E5048093E40480915405D3
:100C300090915505019690935505809354058091A8
:100C40005405909155054B970CF493CF4F5F5F4F30
:100C50004830510509F081CF84E090E09093E3049F
:100C60008093E20483E090E09093E5048093E404B1
:100C700081E090E0909355058093540541E0E42E87
:100C8000F12C012D112D8EC080915605880F809377
:100C90005605809156052091560590E034E09595D3
:100CA00087953A95E1F781709070221F2227221FC5
:100CB00030E08217930721F080915605816003C0D0
:100CC000809156058E7F8093560520915605E091C0
:100CD000E404F091E504E557FE4F80814091E20481
:100CE0005091E30490E002C0959587954A95E2F70C
:100CF00030E08227932780FF17C0E091E404F09151
:100D0000E504E557FE4F20818091E2049091E304D1
:100D1000B801A70104C0440F551F661F771F8A95AD
:100D2000D2F7242B208319C0E091E404F091E5046C
:100D3000E557FE4F20818091E2049091E304570132
:100D4000680104C0AA0CBB1CCC1CDD1C8A95D2F720
:100D5000D601C5018095822380838091E204909121
:100D6000E30401969093E3048093E2048091E2040B
:100D70009091E30408976CF01092E3041092E2045F
:100D80008091E4049091E50401969093E5048093AA
:100D9000E404809154059091550501969093550572
:100DA0008093540580915405909155058559924042
:100DB0000CF46ACFDF91CF911F910F91FF90EF90CC
:100DC000DF90CF90BF90AF9008954091560520914D
:100DD00056058091560530E03595279550E042271D
:100DE00053274170507090E095958795959587951C
:100DF000817090704817590709F18091530520912F
:100E0000520590E0FC01EE0FFF1FE80FF91FE20F03
:100E1000F11DE250FB4F4081209154053091550562
:100E200081E090E0A0E0B0E004C0880F991FAA1F05
:100E3000BB1F2A95D2F7482B408321C080915305D0
:100E40002091520590E0FC01EE0FFF1FE80FF91F03
:100E5000E20FF11DE250FB4F40812091540530918B
:100E6000550581E090E0A0E0B0E004C0880F991F34
:100E7000AA1FBB1F2A95D2F7809584238083809177
:100E8000540590915505019690935505809354050E
:100E9000209156058091560590E0959587959595FA
:100EA000879530E08227932780FF21C080915305EA
:100EB0002091520590E0FC01EE0FFF1FE80FF91F93
:100EC000E20FF11DE250FB4F40812091540530911B
:100ED000550581E090E0A0E0B0E004C0880F991FC4
:100EE000AA1FBB1F2A95D2F7482B408321C08091AF
:100EF00053052091520590E0FC01EE0FFF1FE80F13
:100F0000F91FE20FF11DE250FB4F40812091540583
:100F10003091550581E090E0A0E0B0E004C0880F7A
:100F2000991FAA1FBB1F2A95D2F78095842380831F
:100F300080915405909155050196909355058093A5
:100F400054050895CF93DF931092530510925205E4
:100F500010925605109255051092540581E090E0CC
:100F600045C0C0E0D0E080915605880F80935605BB
:100F7000E0918205F0918305E95AFA4F808190E073
:100F80000C2E02C0959587950A94E2F780FF04C065
:100F900080915605816003C0809156058E7F8093B5
:100FA00056050E94E50680915405909155050897D5
:100FB000A4F01092550510925405809152058F5F50
:100FC0008093520580915205833038F0109252057B
:100FD000809153058F5F809353052196C830D105CA
:100FE00011F6809182059091830501969093830577
:100FF0008093820580918205909183058A970CF4F5
:10100000B0CF80915605880F809356058091560584
:101010008E7F809356050E94E50680915605880FC5
:1010200080935605809156058E7F809356050E94C9
:10103000E506DF91CF9108958091560583FFC6C0E4
:101040008091560586FFC2C004C08091560586FD7A
:10105000C1C080915605880F809356058091560532
:101060008E7F809356058091F00480FFBCC08091F4
:10107000560580FFB8C004C08091560580FDB7C0FA
:10108000809153052091520590E0FC01EE0FFF1F67
:10109000E80FF91FE20FF11DE250FB4F4081209154
:1010A00054053091550581E090E0A0E0B0E004C027
:1010B000880F991FAA1FBB1F2A95D2F780958423FA
:1010C0008083809153058F5F8093530580915205F3
:1010D000882301F5809153058C31E0F0109253057F
:1010E00080915405909155050197909355058093F3
:1010F0005405809154059091550597FF0BC087E0EA
:1011000090E09093550580935405809152058F5F30
:101110008093520580915205813079F48091530576
:101120008C3158F0109253058091540590915505DB
:101130000197909355058093540580915205813015
:10114000A9F4809153058B3189F4809154059091D5
:10115000550504975CF410925305809154059091C5
:10116000550501979093550580935405809154053A
:101170009091550597FF0BC087E090E0909355053F
:1011800080935405809152058F5F80935205809122
:101190005205823009F04CC0809153058B3108F420
:1011A00047C01092530580915405909155050197C1
:1011B0009093550580935405809154059091550561
:1011C00097FF36C083E08093FB0508958091560514
:1011D00083FF3BCF80915605880F80935605809101
:1011E000560581603ECF8091F00480FF45CF80910D
:1011F00053052091520590E0FC01EE0FFF1FE80F10
:10120000F91FE20FF11DE250FB4F40812091540580
:101210003091550581E090E0A0E0B0E004C0880F77
:10122000991FAA1FBB1F2A95D2F7482B408349CF8D
:1012300008958091560587FF19C08091560582FF59
:1012400015C004C08091560582FD14C080915605DA
:101250008E7F809356058091810590E095958795C6
:1012600080938105809181058F7713C08091560509
:1012700087FFE8CF80915605816080935605809165
:10128000810590E0959587958093810580918105F2
:1012900080688093810580915605880F809356055C
:1012A00008958091FD048F5F8093FD048091FD047B
:1012B000883000F11092FD04E0914F01F09150014F
:1012C000E557FE4F80818093E60480914F01909115
:1012D000500101979093500180934F0180914F01ED
:1012E00090915001892B31F48CE291E09093500160
:1012F00080934F01E6E1F0E0DF01AA51BB4F8C91F2
:1013000090E0959587958C939F0121503040F9018D
:10131000EA51FB4F808180FF03C08C91806802C03E
:101320008C918F778C938FEF2F3F380711F0F90155
:10133000E3CF089510927D0110927C0186E591E043
:1013400090937B0180937A0184E0809388010895D3
:10135000AF92BF92CF92DF92EF92FF920F931F93C3
:10136000DF93CF93CDB7DEB7AA970FB6F894DEBF61
:101370000FBECDBF20E030E05E010894A11CB11C7F
:10138000FAE0CF2ED12CCC0EDD1E8E010D5E1F4F4C
:10139000ECE1EE2EF12CEC0EFD1EF901E55AFA4FB0
:1013A0008081F501E20FF31F8083F901ED59FA4FB7
:1013B0008081F601E20FF31F8083F901E559FA4FAE
:1013C0008081F801E20FF31F8083F901ED58FA4F95
:1013D0008081F701E20FF31F80832F5F3F4F28309A
:1013E0003105D9F68FE28CA380917B058DA3809186
:1013F0007C058EA380917D058FA380917E0588A7B3
:1014000019861A8A1B8E19A68B89809331068C89BE
:10141000809332068D89809333068E8980933406BB
:101420008F8980933506888D80933606898D8093C9
:1014300037068A8D809338061092390681E08093B2
:101440008001809381018AE791E063E040E00E949F
:10145000E71B8AE791E060E071E00E94121E8AE7D4
:1014600091E063E047E30E94E71B8AE791E0B8015F
:101470000E94D4268AE791E065E040E00E94E71BE5
:101480008AE791E06AE071E00E94121E8AE791E02B
:1014900065E042E30E94E71B8AE791E0B7010E9402
:1014A000D4268AE791E067E040E00E94E71B8AE7E4
:1014B00091E0B6010E94D4268AE791E067E040E41B
:1014C0000E94E71B8AE791E064E171E00E94121E2E
:1014D0008AE791E067E040E50E94E71B8AE791E038
:1014E000B5010E94D426AA960FB6F894DEBF0FBEAF
:1014F000CDBFCF91DF911F910F91FF90EF90DF90C3
:10150000CF90BF90AF900895AF92BF92CF92DF92ED
:10151000EF92FF920F931F93DF93CF93CDB7DEB778
:10152000AA970FB6F894DEBF0FBECDBF20E030E023
:101530005E010894A11CB11CBAE0CB2ED12CCC0EBC
:10154000DD1E8E010D5E1F4FACE1EA2EF12CEC0E7C
:10155000FD1EF901E65AFA4F8081F501E20FF31FF3
:101560008083F901EE59FA4F8081F601E20FF31FF3
:101570008083F901E659FA4F8081F801E20FF31FE9
:101580008083F901EE58FA4F8081F701E20FF31FD3
:1015900080832F5F3F4F28303105D9F68FE28CA32F
:1015A00080917A058DA380917B058EA380917C0527
:1015B0008FA380917D0588A719861A8A1B8E19A68C
:1015C0008B89809331068C89809332068D89809334
:1015D00033068E89809334068F8980933506888DF3
:1015E00080933606898D809337068A8D80933806DE
:1015F0001092390681E080938001809381018AE70F
:1016000091E063E040E00E94E71B8AE791E060E040
:1016100071E00E94121E8AE791E063E047E30E94B6
:10162000E71B8AE791E0B8010E94D4268AE791E09F
:1016300065E040E00E94E71B8AE791E06AE071E024
:101640000E94121E8AE791E065E042E30E94E71BD8
:101650008AE791E0B7010E94D4268AE791E067E02B
:1016600040E00E94E71B8AE791E0B6010E94D42681
:101670008AE791E067E040E40E94E71B8AE791E097
:1016800064E171E00E94121E8AE791E067E040E5A4
:101690000E94E71B8AE791E0B5010E94D426AA9632
:1016A0000FB6F894DEBF0FBECDBFCF91DF911F9173
:1016B0000F91FF90EF90DF90CF90BF90AF90089583
:1016C000EF92FF920F931F93609118067091190685
:1016D00080911A0690911B0664527C4B8140904089
:1016E0000E94C22828EA3DEF40EE5AE40E942728D3
:1016F00060931C0670931D0680931E0690931F0630
:1017000060911C0670911D0680911E0690911F0627
:101710000E94FD280E94942860932006E0901C06F9
:10172000F0901D0600911E0610911F066091200684
:1017300070E0882777FD8095982F0E94C2289B0132
:10174000AC01C801B7010E94BE2720E030E040E0B4
:1017500057E40E94CB2960931C0670931D0680936A
:101760001E0690931F0660911C0670911D068091C5
:101770001E0690911F0620E030E040E05FE30E94EB
:10178000BF270E94FD280E94942870932206609330
:10179000210683E090E0A0E0B0E0809323069093E0
:1017A0002406A0932506B0932606809123069091E7
:1017B0002406A0912506B0912606BA2FA92F982FAE
:1017C00088278093230690932406A0932506B09340
:1017D000260620912306309124064091250650913B
:1017E00026068091200690E0A0E0B0E0822B932BAB
:1017F000A42BB52B8093230690932406A093250653
:10180000B09326068091230690912406A091250688
:10181000B09126064FE0880F991FAA1FBB1F4A955B
:10182000D1F78093230690932406A0932506B093C6
:1018300026062091230630912406409125065091DA
:1018400026068091210690912206A0E0B0E0822B2E
:10185000932BA42BB52B8093230690932406A0935F
:101860002506B09326068091230690912406A09128
:101870002506B091260634E0880F991FAA1FBB1FCA
:101880003A95D1F78093230690932406A0932506DA
:10189000B0932606609118067091190680911A0679
:1018A00090911B0664587543804090400E94C22866
:1018B00028EA3DEF40EE5AE40E94272860931C0678
:1018C00070931D0680931E0690931F0660911C0660
:1018D00070911D0680911E0690911F060E94FD28A2
:1018E0000E94942860932006E0901C06F0901D064C
:1018F00000911E0610911F066091200670E0882757
:1019000077FD8095982F0E94C2289B01AC01C801E9
:10191000B7010E94BE2720E030E040E057E40E947B
:10192000CB2960931C0670931D0680931E0690932E
:101930001F0660911C0670911D0680911E069091F5
:101940001F0620E030E040E05FE30E94BF270E94D6
:10195000FD280E949428709322066093210682E05D
:1019600090E0A0E0B0E08093270690932806A09333
:101970002906B0932A068091270690912806A09107
:101980002906B0912A06BA2FA92F982F882780936D
:10199000270690932806A0932906B0932A06209143
:1019A0002706309128064091290650912A068091F9
:1019B000200690E0A0E0B0E0822B932BA42BB52B67
:1019C0008093270690932806A0932906B0932A06B1
:1019D0008091270690912806A0912906B0912A06A9
:1019E0000FE0880F991FAA1FBB1F0A95D1F780939C
:1019F000270690932806A0932906B0932A062091E3
:101A00002706309128064091290650912A06809198
:101A1000210690912206A0E0B0E0822B932BA42B0C
:101A2000B52B8093270690932806A0932906B093A0
:101A30002A068091270690912806A0912906B09148
:101A40002A0614E0880F991FAA1FBB1F1A95D1F709
:101A50008093270690932806A0932906B0932A0620
:101A60001F910F91FF90EF900895EF92FF920F93C7
:101A70001F9380918B0590E090932C0680932B060A
:101A800080912B0690912C06A0E0B0E08093180680
:101A900090931906A0931A06B0931B0680918C05AB
:101AA00090E090932C0680932B062091180630919D
:101AB000190640911A0650911B0680912B069091B1
:101AC0002C06982F8827A0E0B0E0820F931FA41F58
:101AD000B51F8093180690931906A0931A06B09329
:101AE0001B0680918D0590E090932C0680932B0629
:101AF000209118063091190640911A0650911B0644
:101B000080912B0690912C06A0E0B0E0DC01992793
:101B10008827820F931FA41FB51F809318069093E8
:101B20001906A0931A06B0931B0680918E0590E0CB
:101B300090932C0680932B0620911806309119065D
:101B400040911A0650911B0680912B0690912C060D
:101B5000A0E0B0E0B82FAA2799278827820F931F0B
:101B6000A41FB51F8093180690931906A0931A0618
:101B7000B0931B06609118067091190680911A06A1
:101B800090911B0664527C4B814090400E94C22879
:101B900028EA3DEF40EE5AE40E94272860931C0695
:101BA00070931D0680931E0690931F0660911C067D
:101BB00070911D0680911E0690911F060E94FD28BF
:101BC0000E94942860932006E0901C06F0901D0669
:101BD00000911E0610911F066091200670E0882774
:101BE00077FD8095982F0E94C2289B01AC01C80107
:101BF000B7010E94BE2720E030E040E057E40E9499
:101C0000CB2960931C0670931D0680931E0690934B
:101C10001F0660911C0670911D0680911E06909112
:101C20001F0620E030E040E05FE30E94BF270E94F3
:101C3000FD280E949428709322066093210683E079
:101C400090E0A0E0B0E08093230690932406A09358
:101C50002506B09326068091230690912406A09134
:101C60002506B0912606BA2FA92F982F8827809392
:101C7000230690932406A0932506B0932606209170
:101C80002306309124064091250650912606809126
:101C9000200690E0A0E0B0E0822B932BA42BB52B84
:101CA0008093230690932406A0932506B0932606DE
:101CB0008091230690912406A0912506B0912606D6
:101CC0001FE0880F991FAA1FBB1F1A95D1F7809399
:101CD000230690932406A0932506B0932606209110
:101CE00023063091240640912506509126068091C6
:101CF000210690912206A0E0B0E0822B932BA42B2A
:101D0000B52B8093230690932406A0932506B093C9
:101D100026068091230690912406A0912506B09175
:101D20002606F4E0880F991FAA1FBB1FFA95D1F76A
:101D30008093230690932406A0932506B09326064D
:101D4000609118067091190680911A0690911B06F1
:101D500064587543804090400E94C22828EA3DEFB5
:101D600040EE5AE40E94272860931C0670931D06DB
:101D700080931E0690931F0660911C0670911D06AD
:101D800080911E0690911F060E94FD280E949428B3
:101D900060932006E0901C06F0901D0600911E0640
:101DA00010911F066091200670E0882777FD8095CE
:101DB000982F0E94C2289B01AC01C801B7010E9464
:101DC000BE2720E030E040E057E40E94CB2960933A
:101DD0001C0670931D0680931E0690931F0660914B
:101DE0001C0670911D0680911E0690911F0620E032
:101DF00030E040E05FE30E94BF270E94FD280E9480
:101E00009428709322066093210682E090E0A0E07F
:101E1000B0E08093270690932806A0932906B093FC
:101E20002A068091270690912806A0912906B09154
:101E30002A06BA2FA92F982F8827809327069093D8
:101E40002806A0932906B0932A06209127063091F0
:101E500028064091290650912A068091200690E09C
:101E6000A0E0B0E0822B932BA42BB52B8093270608
:101E700090932806A0932906B0932A0680912706FE
:101E800090912806A0912906B0912A067FE0880F3C
:101E9000991FAA1FBB1F7A95D1F7809327069093AD
:101EA0002806A0932906B0932A0620912706309190
:101EB00028064091290650912A068091210690918A
:101EC0002206A0E0B0E0822B932BA42BB52B8093AD
:101ED000270690932806A0932906B0932A0680919E
:101EE000270690912806A0912906B0912A0664E061
:101EF000880F991FAA1FBB1F6A95D1F780932706E9
:101F000090932806A0932906B0932A061F910F915B
:101F1000FF90EF9008958091100690911106019620
:101F2000909311068093100685E00E945E23892B12
:101F300021F080918901806803C0809189018F77A9
:101F40008093890180918A018F5F80938A018091BB
:101F50008A01883009F5E0914D01F0914E018091A0
:101F60008901E557FE4F808380914D0190914E018C
:101F7000019790934E0180934D0180914D01909176
:101F80004E01892B31F48CE291E090934E018093C5
:101F90004D0110928A0107C08091890190E09595CA
:101FA00087958093890181E08093FD050895809154
:101FB00010069091110601969093110680931006D9
:101FC00080910506909106060197909306068093EE
:101FD00005068091FE05843021F08091FE05853054
:101FE00009F510920C0610920B0680910D06815097
:101FF00080930D0686E00E945E23019719F486E027
:1020000060E002C086E061E00E940A238091FE0544
:10201000853041F486E00E945E23019719F486E042
:102020008093FE058091FE05873029F08091FE05A2
:10203000883009F070C080910B0690910C060196D3
:1020400090930C0680930B0680910B0690910C06E2
:10205000803691055CF010920C0610920B06809170
:102060000A068F5F80930A0680910A06E091E004D9
:10207000F091E104E557FE4F80812091E204309118
:10208000E30490E002C0959587952A95E2F780FFDA
:1020900003C086E061E002C086E060E00E940A239F
:1020A0008091E2049091E30401969093E30480937D
:1020B000E2048091E2049091E3040897D1F4109235
:1020C000E3041092E2048091E0049091E10401960F
:1020D0009093E1048093E0048091E0049091E10406
:1020E0008355934034F081E090E09093E104809335
:1020F000E0048091FE05883071F42091DE04309177
:10210000DF048091E0049091E1042817390719F465
:1021100089E08093FE0581E08093000683E060E023
:102120000E940A2308958FE190E029C08091120651
:1021300090911306A0911406B091150620911606F1
:102140003091170604C0B595A795979587952A9560
:10215000D2F780FF03C08AE061E002C08AE060E05D
:102160000E940A2387E061E00E940A2387E060E082
:102170000E940A238091160690911706019790936A
:10218000170680931606809116069091170697FF02
:10219000CDCF8CE061E00E940A238CE060E00E94D9
:1021A0000A238AE060E00E940A23089585EF94E202
:1021B000A0E0B0E08093120690931306A09314065B
:1021C000B09315060E94931082E990EDA5E6B1E068
:1021D0008093120690931306A0931406B0931506ED
:1021E0000E94931083E990ECACE4BAE2809312066B
:1021F00090931306A0931406B09315060E949310B3
:1022000084E194ECA5E4B0E4809312069093130665
:10221000A0931406B09315060E9493108091230694
:1022200090912406A0912506B0912606809312066F
:1022300090931306A0931406B09315060E94931072
:10224000089582E990EDA5E7B0E08093120690939F
:102250001306A0931406B09315060E949310809164
:10226000270690912806A0912906B0912A0680930E
:10227000120690931306A0931406B09315060E94BD
:102280009310089581E190E5A7E5B0E080931206F0
:1022900090931306A0931406B09315060E94931012
:1022A00083E990ECACE4BAE28093120690931306B3
:1022B000A0931406B09315060E94931080912306F4
:1022C00090912406A0912506B091260680931206CF
:1022D00090931306A0931406B09315060E949310D2
:1022E00085EF94E2A0E0B0E080931206909313068D
:1022F000A0931406B09315060E94931084E194EC09
:10230000A5E4B0E48093120690931306A0931406FC
:10231000B09315060E94931082E990EDA5E6B1E016
:102320008093120690931306A0931406B09315069B
:102330000E9493108FE090E0AEE0B0E08093120630
:1023400090931306A0931406B09315060E94931061
:1023500086E09EE0A7E0B5E0809312069093130616
:10236000A0931406B09315060E94931089EE91E392
:10237000A2E0B0E08093120690931306A093140697
:10238000B09315060E9493108AE397E4A6E9B2E39E
:102390008093120690931306A0931406B09315062B
:1023A0000E9493108BE390E0A0E0B0E080931206CF
:1023B00090931306A0931406B09315060E949310F1
:1023C0008CE091E0A0E0B0E08093120690931306B9
:1023D000A0931406B09315060E9493108DE090E030
:1023E000A0E0B0E08093120690931306A093140629
:1023F000B09315060E949310089580E480938B0596
:1024000088E780938C0587EE80938D0589E1809322
:102410008E050E94350D0E94421180E00E948221AB
:1024200080E06BE87FE043E050E00E945F21089588
:1024300080E00E94822180E06BE87FE043E050E092
:102440000E945F2181E00E948221809108068E7F98
:1024500080930806809108068D7F8093080688E0A7
:1024600060E00E940A238DE060E00E940A230E943F
:10247000D6108CE291E090934E0180934D01109222
:10248000FD041092FB051092F8051092F9051092C8
:102490000A061092090681E08093FE051092FF055E
:1024A0008093FC050895CF93DF9380ED8093BF0563
:1024B0000E94A503C1E0D0E009C0FE01E254FA4F3A
:1024C00060818FE098E00E94332521968091F60587
:1024D0009091F7058C179D0784F7DF91CF910895B0
:1024E000FF920F931F938091F4048A3A09F050C031
:1024F0008091F3048A3A09F04BC08091F2048E3641
:1025000009F046C08091F1048A3009F041C082E0B0
:102510008093FB05109252051092530587E090E0DE
:1025200090935505809354058FEF80935605109234
:10253000FA05809151018F5F80935101A3E0FA2E3B
:10254000F092C0051092C10585E18093C2051092FA
:10255000C3051092C40506E010E01093F705009340
:10256000F6050E945312F092C0051092C10586E153
:102570008093C205809151018093C3058091FA0533
:102580008093C4051093F7050093F6050E9453123B
:102590001F910F91FF9008951092530510925205CC
:1025A00010925605109283051092820514C1109264
:1025B00081058091530590E020915205FC01EE0FBA
:1025C000FF1FE80FF91FE20FF11DE250FB4F808162
:1025D00086FF04C080915605806803C0809156052F
:1025E0008F77809356050E9419098091530590E0DA
:1025F00020915205FC01EE0FFF1FE80FF91FE20FBB
:10260000F11DE250FB4F808184FF04C0809156058C
:10261000806803C0809156058F77809356050E948D
:1026200019098091530590E020915205FC01EE0FAD
:10263000FF1FE80FF91FE20FF11DE250FB4F8081F1
:1026400082FF04C080915605806803C080915605C2
:102650008F77809356050E9419098091530590E069
:1026600020915205FC01EE0FFF1FE80FF91FE20F4A
:10267000F11DE250FB4F808180FF04C08091560520
:10268000806803C0809156058F77809356050E941D
:102690001909809152058F5F8093520580915205F0
:1026A000833038F010925205809153058F5F8093EC
:1026B00053058091530590E020915205FC01EE0FE7
:1026C000FF1FE80FF91FE20FF11DE250FB4F808161
:1026D00086FF04C080915605806803C0809156052E
:1026E0008F77809356050E9419098091530590E0D9
:1026F00020915205FC01EE0FFF1FE80FF91FE20FBA
:10270000F11DE250FB4F808184FF04C0809156058B
:10271000806803C0809156058F77809356050E948C
:1027200019098091530590E020915205FC01EE0FAC
:10273000FF1FE80FF91FE20FF11DE250FB4F8081F0
:1027400082FF04C080915605806803C080915605C1
:102750008F77809356050E9419098091530590E068
:1027600020915205FC01EE0FFF1FE80FF91FE20F49
:10277000F11DE250FB4F808180FF04C0809156051F
:10278000806803C0809156058F77809356050E941C
:102790001909809152058F5F8093520580915205EF
:1027A000833038F010925205809153058F5F8093EB
:1027B0005305E0918205F091830580918105E95AE6
:1027C000FA4F8083809182059091830501969093C2
:1027D0008305809382058091820590918305899776
:1027E0000CF4E5CE84E08093FB058FE28093C00576
:1027F0001092C10587E18093C205809151018093B9
:10280000C3058091FA058093C4051092C505109206
:10281000C605109283051092820517C0A09182050B
:10282000B0918305E0918205F0918305E95AFA4F52
:102830008081A953BA4F8C93809182059091830532
:1028400001969093830580938205809182059091F3
:10285000830589971CF30E94840A82E390E0909399
:10286000F7058093F6050E9453120895809187051D
:10287000813109F040C08093C0051092C10581E903
:102880008093C2051092C30594E59093C40583E537
:102890008093C50580E58093C60588E38093C705CE
:1028A0008EE48093C8059093C90588E48093CA0597
:1028B00080E28093CB058093CC0584E48093CD05A2
:1028C00086E58093CE058DE28093CF059093D00569
:1028D00082E58093D10588E58093D20584E190E07C
:1028E0009093F7058093F6050E94531281E0809340
:1028F000FE058093FC05809187058231E1F485E037
:102900008093C0051092C10582E98093C20583E1DE
:102910008093C30589E08093C40580E18093C50559
:1029200081E08093C60588E090E09093F70580935E
:10293000F6050E945312809187058431D9F5809164
:102940008805803C91F480918A05809301068091EE
:102950008B058093020680918C05809303068091FD
:102960008D05809304060E94FD1180918805813CAD
:1029700071F480E00E9482210E94350D80E06BE8B6
:102980007FE043E050E00E945F210E94421182E01C
:102990008093C0051092C10584E98093C20586E04A
:1029A0008093C30585E090E09093F7058093F6054A
:1029B0000E945312809187058031D1F49091850552
:1029C0009230B1F480918805809307069093C005FA
:1029D0001092C10580E98093C20586E08093C3050B
:1029E00085E090E09093F7058093F6050E945312DE
:1029F00080918705803169F580918505813049F5A1
:102A000088E08093C0051092C10580E98093C205DB
:102A100087E48093C305809108068093C405809164
:102A2000FC058093C50585E18093C6058CEF8093F6
:102A3000C705809109068093C80580910A06809396
:102A4000C9058BE090E09093F7058093F6050E940E
:102A5000531280918705863139F486E060E00E9448
:102A60000A2381E08093FF0580918705873161F516
:102A70008091880580935101809189058093FA05A2
:102A800021E030E0F901E557FA4F8081F901E95A78
:102A9000FA4F80832F5F3F4F2A32310599F70E940A
:102AA000A80986E590E09093DF048093DE0481E03E
:102AB00090E09093E1048093E0040E94A2070E94BA
:102AC000E30382E08093FF0580918705893109F057
:102AD0003EC010921106109210068091F9058F5F8A
:102AE0008093F9058091F905853110F01092F90570
:102AF00028E030E041E050E0E091DE04F091DF04B6
:102B0000D901AC57BA4F8C91E557FE4F8083809125
:102B1000DE049091DF0401969093DF048093DE043D
:102B20008091DE049091DF048355934024F050930C
:102B3000DF044093DE042F5F3F4F24313105E1F67F
:102B40008091FF05823019F483E08093FF05809126
:102B500087058A3109F04DC18091DE049091DF0430
:102B600001979093DF048093DE048091DE049091BE
:102B7000DF04892B31F482E593E09093DF048093A6
:102B8000DE048091DE049091DF0401979093DF04CE
:102B90008093DE048091DE049091DF04892B31F470
:102BA00082E593E09093DF048093DE048091DE045D
:102BB0009091DF0401979093DF048093DE0480916D
:102BC000DE049091DF04892B31F482E593E0909349
:102BD000DF048093DE04E091DE04F091DF04E5572A
:102BE000FE4F85E580838091DE049091DF0401969D
:102BF0009093DF048093DE048091DE049091DF04E3
:102C00008355934034F081E090E09093DF0480930B
:102C1000DE04E091DE04F091DF04E557FE4F85E528
:102C200080838091DE049091DF0401969093DF040D
:102C30008093DE048091DE049091DF0483559340FD
:102C400034F081E090E09093DF048093DE04E09123
:102C5000DE04F091DF04E557FE4F85E58083809127
:102C6000DE049091DF0401969093DF048093DE04EC
:102C70008091DE049091DF048355934034F081E02D
:102C800090E09093DF048093DE04E091DE04F09105
:102C9000DF04E557FE4F85E580838091DE04909147
:102CA000DF0401969093DF048093DE048091DE04BC
:102CB0009091DF048355934034F081E090E090934D
:102CC000DF048093DE04E091DE04F091DF04E55739
:102CD000FE4F88EC80838091DE049091DF040196A2
:102CE0009093DF048093DE048091DE049091DF04F2
:102CF0008355934034F081E090E09093DF0480931B
:102D0000DE04E091DE04F091DF04E557FE4F8AE730
:102D100080838091DE049091DF0401969093DF041C
:102D20008093DE048091DE049091DF04835593400C
:102D300034F081E090E09093DF048093DE04E09132
:102D4000DE04F091DF04E557FE4F10828091DE042F
:102D50009091DF0401969093DF048093DE048091CC
:102D6000DE049091DF048355934034F081E090E0DD
:102D70009093DF048093DE04E091DE04F091DF04A1
:102D8000E557FE4F10828091DE049091DF0401969A
:102D90009093DF048093DE048091DE049091DF0441
:102DA0008355934034F081E090E09093DF0480936A
:102DB000DE04E091DE04F091DF04E557FE4F10825F
:102DC0008091DE049091DF0401969093DF0480935C
:102DD000DE048091DE049091DF048355934034F04B
:102DE00081E090E09093DF048093DE0484E08093A0
:102DF000FF05809187058F31E1F590918805903C22
:102E0000D1F486E08093C0051092C1058FE98093CC
:102E1000C2059093C3051092C4051092C505109287
:102E2000C6051092C70589E090E09093F70580935E
:102E3000F6050E94531290918805913CD1F486E0EA
:102E40008093C0051092C1058FE98093C2059093CD
:102E5000C3051092C4051092C5051092C6051092C4
:102E6000C70589E090E09093F7058093F6050E94EE
:102E7000531210928405109285051092BD05109290
:102E8000BC05089583E18093C0051092C10589E1D6
:102E90008093C205809151018093C3058091FA050A
:102EA0008093C40588EE8093C50583E08093C605B2
:102EB00025E130E04EE150E0FA01E21BF30BD901CD
:102EC000AA51BB4F8C91E254FA4F8083215030407D
:102ED0002930310589F71092D3051092D40586E187
:102EE00090E09093F7058093F6050E9453120895A1
:102EF00083E08093C0051092C1058AE18093C205EA
:102F0000809151018093C3058091FA058093C40597
:102F100086E090E09093F7058093F6050E945312A7
:102F200008950F931F93CF93DF9320912D06309137
:102F30002E0640912F0650913006809118069091F0
:102F40001906A0911A06B0911B06281739074A07DF
:102F50005B0709F44EC080E00E9482210E94600B52
:102F60000E94421180E06BE87FE043E050E00E9465
:102F70005F218091180690911906A0911A06B091D0
:102F80001B0680932D0690932E06A0932F06B093D8
:102F900030068AE791E060E045E00E94E71B82E0AE
:102FA0008093800181E08093810160912D06709172
:102FB0002E0680912F06909130060E94C22820E0B4
:102FC00034E244E759E40E942728AB01BC018AE7B8
:102FD00091E023E030E00E94BB278AE791E060E0C7
:102FE0004AE50E94E71B8AE791E066E171E00E94F2
:102FF000121E8FE098E00E94C624181619060CF5E0
:103000000091BC051091BD058FE098E00E94FA2464
:103010000C571A4FF80180838091BC059091BD0533
:1030200001969093BD058093BC058091BC0590915D
:10303000BD05C89734F087E390E09093BD05809379
:10304000BC0580918405803D21F01092BD05109251
:10305000BC0580918405803D99F48091BC059091D8
:10306000BD0505976CF02091BC053091BD058091A0
:10307000850590E004968217930714F40E94361495
:1030800080910006813009F045C02091DE04309126
:10309000DF048091E0049091E1048217930784F4A7
:1030A0008091DE049091DF042091E0043091E104EE
:1030B000821B930B6CE070E00E94652A6093090606
:1030C0002091DE043091DF048091E0049091E104CE
:1030D0002817390794F48091DE049091DF04209141
:1030E000E0043091E1048E5A9C4F821B930B6CE0FC
:1030F00070E00E94652A609309062091DE043091F9
:10310000DF048091E0049091E1042817390711F45D
:10311000109209068091FE05882309F4ECC0809185
:10312000FE05813009F058C08091FF05882309F41D
:1031300053C08AEF90E09093500180934F018CE24E
:1031400091E090934E0180934D0180E00E94822196
:1031500081E00E948221809108068E7F809308067C
:103160008091080682608093080688E061E00E94F2
:103170000A238DE061E00E940A230E94211180E071
:1031800067ED7FE042E050E00E945F2180910306FE
:1031900025E0829FC00111249093060680930506C6
:1031A00040910506509106068091040690E02BEFB1
:1031B00034E0BC01629FC001639F900D729F900D2F
:1031C0001124840F951F909306068093050682E0D4
:1031D0008093FE058093FC058091FE05823049F4C2
:1031E0008091050690910606059718F483E0809378
:1031F000FE059091FE05933061F48091FF058230C9
:1032000040F080E480930D0684E08093FE05909367
:10321000FC058091FE05843039F480910D068230E2
:1032200018F485E08093FE058091FE05863031F428
:1032300087E08093FE0585E08093FC058091FE0584
:10324000873009F045C08091100690911106815C8D
:10325000924110F00E941812809109068530D0F436
:103260008091E0049091E104CC979093E1048093E5
:10327000E0048091E0049091E1041816190654F0DE
:103280008091E0049091E1048E5A9C4F9093E10468
:103290008093E004809109068334D0F08091DE04AD
:1032A0009091DF04CC979093DF048093DE048091AB
:1032B000DE049091DF041816190654F08091DE04A4
:1032C0009091DF048E5A9C4F9093DF048093DE042C
:1032D0009091FE05973049F48091FF05843029F4E0
:1032E00088E08093FE059093FC058091FE0589306F
:1032F00011F40E9418128091FB058630C0F52091D0
:103300004D0130914E0180914F01909150018217F3
:10331000930794F480914F019091500120914D01B9
:1033200030914E01845D9E4F821B930B8B3F910524
:103330001CF081E08093FD0520914F0130915001F8
:1033400080914D0190914E018217930784F48091F2
:103350004F019091500120914D0130914E01821BFF
:10336000930B8B3F91051CF081E08093FD058091CC
:10337000FD05813009F04AC10E9451098091FB0589
:103380008823D9F49091FD059130B9F48091F4042B
:103390008A3A99F48091F3048A3A79F48091F2049C
:1033A0008A3A59F48091F1048A3A39F49093FB05F2
:1033B000809108068160809308068091FB0581302A
:1033C00031F48091FD05813011F40E9470128091DA
:1033D000FB05823061F48091FD05813041F40E944B
:1033E0001C081092FE0583E061E00E940A23809190
:1033F000FB05833031F48091FD05813011F40E948A
:10340000CC128091FB05843039F48091FD05813028
:1034100019F485E08093FB058091FB058530D1F49C
:103420008091FD058130B1F405C00E945109809161
:10343000F8058F5F8093F8058091F8058131A8F336
:1034400086E08093FB051092F80584E18093F905EE
:103450001092FD058091FB05863009F0D7C0809160
:10346000FD05813009F0D2C08091F8058F5F80930F
:10347000F8058091F805823008F44FC08091F80576
:10348000893108F04AC020914F013091500180915C
:103490004D0190914E0182179307CCF480914F011A
:1034A0009091500120914D0130914E01821B930B60
:1034B00045976CF0C1E0D0E00E9451098091F80579
:1034C0008F5F8093F8052196C132D105A9F720912D
:1034D0004F013091500180914D0190914E0128177C
:1034E0003907DCF480914F019091500120914D01FA
:1034F00030914E01845D9E4F821B930B45976CF07B
:10350000C1E0D0E00E9451098091F8058F5F80935F
:10351000F8052196C132D105A9F78091F8058934C3
:10352000E1F48091F2048535C1F48091F104853590
:10353000A1F48091F004853581F48091EF04853504
:1035400061F48091EE04883C41F48091ED048A3767
:1035500021F40E9418120E9478178091F905843195
:10356000A1F48091F805823480F08091F1048535D2
:1035700061F48091F0048D3241F48091EF04863142
:1035800021F41092FD050E9451098091F9058431C2
:1035900011F58091F8058934F1F48091F2048535B4
:1035A000F1F58091F1048D32D1F58091F0048631EE
:1035B000B1F511C08091F1048D3221F08091F004B9
:1035C000863191F585E58093F2048DE28093F104D4
:1035D00086E18093F0048091F805893431F480917C
:1035E000F9058093FA050E9442178091F80580360C
:1035F00068F01092F8058091F9058F5F8093F905C6
:103600008091F905853110F01092F9051092FD05B1
:1036100010920006DF91CF911F910F910895809134
:10362000F204853539F6CECF0E9418120E94781721
:10363000D2CFEF92FF920F931F930AE711E0C801D8
:103640000E94261EC8010E94E31DC80160E045E0FB
:103650000E94E71B82E0F82EF0928001EE24E394B2
:10366000E0928101C8016AE171E00E94121E83E0CC
:1036700080938001F0928101C80163E040E00E94E4
:10368000E71BC80166E271E00E94121EE092800111
:10369000F0928101C80167E045E00E94E71BC80184
:1036A0006EE271E00E94121E68EE73E080E090E02E
:1036B0000E943722C8010E94E31D82E060E00E9460
:1036C000CB2287E061E00E94CB2285E060E00E948F
:1036D000CB2286E061E00E94CB228AE061E00E947A
:1036E000CB228CE061E00E94CB2288E061E00E9466
:1036F000CB228DE061E00E94CB2283E061E00E945A
:10370000CB2287E060E00E940A238CE060E00E9408
:103710000A238AE060E00E940A2388E060E00E94B9
:103720000A238DE061E00E940A230FE018E0C8013F
:1037300040E052EC61E070E00E943F24C8010E942A
:1037400023250E94FD118DE061E00E940A231F9154
:103750000F91FF90EF9008950F931F938C0180E8D5
:1037600096E00E94311FF80113861F910F91089572
:10377000FC018585882321F480E896E00E94311FB2
:1037800008951F93CF93DF93EC01162F8B85882329
:1037900011F08F3181F41B8680E896E00E94311F82
:1037A00080E896E06CE370E00E946C1E80E896E092
:1037B0006C850E94EE1E80E896E0612F0E94EE1E4E
:1037C0008B858F5F8B87DF91CF911F9108950F932A
:1037D0001F938C016770FC016583842F8F7784832E
:1037E000138614864F70C801642F0E94C11BF80114
:1037F000648165956595659565956061C8010E94D0
:10380000C11BF8016581606BC8010E94C11BC80122
:103810000E94B81B1F910F910895BF92CF92DF9223
:10382000EF92FF920F931F93CF93DF93EC017B01F5
:103830006A0181E08D8700E010E0BB24B3941FC0D3
:10384000F70160816A3069F41D86CE010E94B81BC1
:103850006D818E81680FCE0140E00E94E71BBD861E
:1038600009C06D3039F0E881F9810190F081E02DD7
:10387000CE0109950894E11CF11C0F5F1F4F0C1538
:103880001D05F0F21D86CE010E94B81BC601DF9116
:10389000CF911F910F91FF90EF90DF90CF90BF904D
:1038A00008952F923F924F925F926F927F928F92E4
:1038B0009F92AF92BF92CF92DF92EF92FF920F93BF
:1038C0001F93CF93DF937C016D3009F455C16A30AB
:1038D00039F4FC0165818681680FC70140E04AC167
:1038E0006E3229F06A3319F005E0702E02C013E041
:1038F000712EF7018680F1E08F1659F5F70184816A
:103900008B5F8483138680E4848785E0689F8001D1
:10391000112408531E4FE801FE016491C7010E9463
:10392000C11B21969E01201B2715B0F310E009C092
:10393000F70184818F5F8483C70160E00E94C11B0F
:103940001F5FF7018781181798F3C7010E94B81B02
:1039500013C1862F80538A3008F023C1282D30E010
:10396000F901EE0FFF1FE75BFB4F859194910097E4
:1039700009F417C1E62FF0E0F097EE0FFF1FE80FF4
:10398000F91F45915491F70175809480C901880F02
:10399000991F880F991F682E680CF8E08F1611F494
:1039A00077E0872E6A01AA2460E4562E51C0AA202F
:1039B00031F06A2D670DC701492D0E94E71BF70101
:1039C00013865486BB2432C0E6012196F601849109
:1039D000982F907C5FE3D52ED822903489F4FE0195
:1039E000CD0DD11D08C08F010F5F1F4F6491C7011E
:1039F0000E94C11BF801EC17FD07A9F7EF0114C0E5
:103A0000992311F400E007C0903C11F40FEF03C0BC
:103A1000FE010491219610E005C0C701602F0E94AD
:103A2000C11B1F5F1D15C8F3BD0C6E01B61460F2FB
:103A3000F7018085882359F410E005C0C70160E0D4
:103A40000E94C11B1F5FF70187811817B8F3A39469
:103A5000A81408F4ACCFC7010E94B81BF7018781F6
:103A6000980E868125E0829FC0011124980EC7011F
:103A7000672D492D7FC0292D30E043E0220F331FF1
:103A80004A95E1F7822F90E06C2D70E00E94512A58
:103A9000C10102C0880F991F6A95E2F7682E6C2D4C
:103AA00070E0CB0133E0880F991F3A95E1F7861B50
:103AB000970B821B91090E94652A8111C82E9920BB
:103AC00031F0692D650DC701482D0E94E71BF701F4
:103AD00013864486E501DD24FE01E859FD4F64911B
:103AE000F7015681362D2C2D00E081E0432F46232F
:103AF00090E00BC04111082B880F215019F4330FAF
:103B0000252F05C0882329F09F5F951798F38823F8
:103B100069F710E005C0C701602F0E94C11B1F5F3D
:103B2000F70186811817B8F3D3942196D714A0F221
:103B30008085882359F410E005C0C70160E00E9429
:103B4000C11B1F5FF70187811817B8F39394F70122
:103B5000C6809C1408F48FCFC7010E94B81BF701E0
:103B60008781880E8681789E802D1124880EC7015A
:103B7000652D482D0E94E71B81E090E0DF91CF91F9
:103B80001F910F91FF90EF90DF90CF90BF90AF907B
:103B90009F908F907F906F905F904F903F902F906D
:103BA0000895F7015580848085E0689F50011124B5
:103BB00020E63FEFA20EB31E992491E0292E312C6E
:103BC00080E4482EC4CF0F931F93CF93DF93EC0173
:103BD0001B861C860BE514E0F8016491CE010E945F
:103BE000C11B0F5F1F4FF4E001361F07A9F7CE017D
:103BF0000E94AC1B80E48C8700E010E0CE0160E006
:103C00000E94C11B0F5F1F4F84E000301807B1F7FF
:103C1000CE010E94B81B1C821D82DF91CF911F91A3
:103C20000F910895CF93DF93DB010D900020E9F70A
:103C30001197A61BB70BEC01E881F9810280F38193
:103C4000E02DAD010995DF91CF9108950F931F935A
:103C5000CF93DF93EC011C821D8281E08E838F83E2
:103C6000888780E896E00E94351F1D868CE080934F
:103C7000B8008E8561E00E94CB228E8561E00E94B3
:103C80000A2361E070E080E090E00E9437228E8598
:103C900060E00E940A236AE070E080E090E00E9409
:103CA00037228E8561E00E940A231B861C8601E66E
:103CB00014E0F8016491CE010E94C11B0F5F1F4FF9
:103CC000F4E00A371F07A9F7CE010E94B81BDF9165
:103CD000CF911F910F91089581E080937F066093AB
:103CE0005C0610927D0610927E06089520915B0678
:103CF00030E080915A06281B3109C901089540918E
:103D00005A0680915B06481718F02FEF3FEF0AC064
:103D1000E42FF0E0E65CF94F8081282F30E04F5F20
:103D200040935A06C9010895E0915A0680915B06B6
:103D3000E81718F0EFEFFFEF06C0F0E0E65CF94F90
:103D40008081E82FF0E0CF01089508951092830656
:103D50001092820688EE93E0A0E0B0E080938406A3
:103D600090938506A0938606B09387068EE591E032
:103D700090938106809380060895CF92DF92EF9210
:103D8000FF920F931F93CF93DF937C016B018A0106
:103D900080917F068823A1F0C0E0D0E00DC0D7015C
:103DA000ED91FC91D601AC0FBD1F0190F081E02D8B
:103DB000C7016C9109952196C017D10780F304C003
:103DC000CB01642F0E94951FC801DF91CF911F91F5
:103DD0000F91FF90EF90DF90CF900895DF93CF93F6
:103DE0000F92CDB7DEB7FC01698380917F068823EF
:103DF000C9F080917E06803238F081E090E09383B4
:103E0000828320E030E015C080917D06E82FF0E04D
:103E1000E35AF94F998190838F5F80937D06809359
:103E20007E0605C0CE01019661E00E94951F21E04B
:103E300030E0C9010F90CF91DF9108950F93062FC5
:103E400080915C066DE576E040917E0621E00E945F
:103E5000401F10927D0610927E0610927F060F91F1
:103E6000089561E00E941E1F089510925A06109254
:103E70005B0610927D0610927E060E9441210895F5
:103E80000F931F93582F122F413210F081E04AC038
:103E900080918C068823E1F782E080938C06009362
:103EA0008E068FEF8093F9061092B4064093B50604
:103EB000A4E9B6E0FB0102C081918D938E2F861B91
:103EC0008417D0F310928D0680918D06550F852BA7
:103ED00080938D0680918F06813041F410928F0679
:103EE00080918D068093BB0085EC01C085EE8093A8
:103EF000BC00112321F080918C068230E1F3809187
:103F0000F9068F3F11F480E00DC08091F9068032F0
:103F100011F482E007C08091F906803311F084E04B
:103F200001C083E01F910F910895482F613210F076
:103F300081E0089580918C06843011F082E008952C
:103F40006093D706A6EBB6E0842F9C01F90102C06E
:103F500081918D938E2F841B8617D0F380E0089576
:103F60001F920F920FB60F9211242F933F934F93EE
:103F70005F936F937F938F939F93AF93BF93EF93D1
:103F8000FF938091B90090E0887F90708036910512
:103F900009F4F2C081369105CCF58832910509F417
:103FA0007BC089329105B4F48031910509F46FC06A
:103FB000813191053CF4009709F447C1089709F055
:103FC0004FC165C08831910509F466C0809709F03A
:103FD00047C182C08034910509F4A4C081349105A1
:103FE00044F48033910509F482C0C89709F038C1C0
:103FF00089C08035910509F489C08835910509F497
:1040000096C08834910509F02BC1AEC0883991055E
:1040100009F413C189399105ECF48837910509F445
:10402000ABC0893791054CF48836910509F4A4C0DA
:104030008037910509F014C19FC08838910509F4B3
:10404000FCC08039910509F49DC08038910509F0C4
:1040500007C198C0803B910509F4C6C0813B91051A
:104060004CF4803A910509F49FC0883A910509F013
:10407000F7C0BAC0803C910509F4E3C0883C9105C3
:1040800009F4DFC0883B910509F0EAC0C2C0809105
:104090008D068093BB00CFC09091B4068091B50689
:1040A000981768F49091B406E92FF0E0EC56F94FB8
:1040B00080818093BB009F5F9093B406BCC08091C9
:1040C0008E06882309F44BC085ED8093BC00809157
:1040D000BC0084FDFCCFC2C080E28093F90685ED70
:1040E0008093BC008091BC0084FDFCCFB7C080E30E
:1040F0008093F90685ED8093BC008091BC0084FD1F
:10410000FCCFACC088E38093F9069BC08091B406D5
:104110009091BB00E82FF0E0EC56F94F90838F5F51
:104120008093B4069091B4068091B50682C08091C8
:10413000B4069091BB00E82FF0E0EC56F94F908365
:104140008F5F8093B40680918E06882341F085EDC1
:104150008093BC008091BC0084FDFCCF7FC081E0D7
:1041600080938F0684EA6EC085ED8093BC008091B9
:10417000BC0084FDFCCF72C083E080938C0610925B
:10418000F80659C08091F806803208F056C0809138
:10419000F8069091BB00E82FF0E0E852F94F9083C9
:1041A0008F5F8093F80647C08091F806803230F424
:1041B000E091F806F0E0E852F94F108285ED809327
:1041C000BC008091BC0084FDFCCF10928C066091F5
:1041D000F806E0919206F091930688ED96E070E083
:1041E00009951092F8062DC084E080938C061092F9
:1041F000D6061092D706E0919006F09191060995A7
:104200008091D706882329F481E08093D706109205
:10421000B6069091D606E92FF0E0EA54F94F808176
:104220008093BB009F5F9093D6069091D6068091B5
:10423000D706981710F485EC01C085E88093BC0080
:104240000FC085EC8093BC0009C01092F90685ED83
:104250008093BC008091BC0084FDFCCF10928C0642
:10426000FF91EF91BF91AF919F918F917F916F914E
:104270005F914F913F912F910F900FBE0F901F9024
:10428000189510928C0681E080938E0610928F060E
:1042900082E161E00E940A2383E161E00E940A2337
:1042A000E9EBF0E080818E7F808380818D7F808349
:1042B00088E48093B80085E48093BC000895823040
:1042C00000F5E82FF0E0EE0FFF1FE650F94F718385
:1042D0006083882319F08130A1F408C080916900BF
:1042E0008C7F842B80936900E89A089580916900FF
:1042F000440F551F440F551F837F842B8093690003
:10430000E99A0895823080F4882319F0813021F4ED
:1043100002C0E89801C0E998E82FF0E0EE0FFF1F17
:10432000E650F94F1182108208951F920F920FB636
:104330000F9211242F933F934F935F936F937F932B
:104340008F939F93AF93BF93EF93FF938091FA0660
:104350009091FB06892B29F0E091FA06F091FB067B
:104360000995FF91EF91BF91AF919F918F917F91AF
:104370006F915F914F913F912F910F900FBE0F90D2
:104380001F9018951F920F920FB60F9211242F9322
:104390003F934F935F936F937F938F939F93AF93CD
:1043A000BF93EF93FF938091FC069091FD06892BBC
:1043B00029F0E091FC06F091FD060995FF91EF913F
:1043C000BF91AF919F918F917F916F915F914F912D
:1043D0003F912F910F900FBE0F901F9018951F9235
:1043E0000F920FB60F9211242F933F938F939F93A9
:1043F000AF93BF938091020790910307A0910407A8
:10440000B0910507309106070196A11DB11D232F1C
:104410002D5F2D3720F02D570196A11DB11D209342
:1044200006078093020790930307A0930407B093B5
:1044300005078091FE069091FF06A0910007B091BC
:1044400001070196A11DB11D8093FE069093FF0602
:10445000A0930007B0930107BF91AF919F918F91F7
:104460003F912F910F900FBE0F901F9018959B01B9
:10447000AC017FB7F8948091FE069091FF06A09161
:104480000007B091010766B5A89B05C06F3F19F002
:104490000196A11DB11D7FBFBA2FA92F982F882784
:1044A000860F911DA11DB11D62E0880F991FAA1FE3
:1044B000BB1F6A95D1F7BC012DC0FFB7F89480915E
:1044C000FE069091FF06A0910007B0910107E6B5A6
:1044D000A89B05C0EF3F19F00196A11DB11DFFBFBC
:1044E000BA2FA92F982F88278E0F911DA11DB11DBE
:1044F000E2E0880F991FAA1FBB1FEA95D1F7861B20
:10450000970B885E9340C8F22150304040405040A5
:1045100068517C4F211531054105510571F608950B
:10452000789484B5826084BD84B5816084BD85B58E
:10453000826085BD85B5816085BDEEE6F0E0808155
:1045400081608083E1E8F0E0108280818260808376
:10455000808181608083E0E8F0E0808181608083F9
:10456000E1EBF0E0808184608083E0EBF0E080812B
:1045700081608083EAE7F0E08081846080838081CD
:104580008260808380818160808380818068808375
:104590001092C1000895CF93DF93482F50E0CA01D5
:1045A0008953994FFC0134914D54594FFA0184912C
:1045B000882369F190E0880F991FFC01EB56F94FB1
:1045C000A591B491FC01E156F94FC591D4916623B0
:1045D00051F42FB7F8948C91932F909589238C9355
:1045E000888189230BC0623061F42FB7F8948C91D5
:1045F000932F909589238C938881832B88832FBF59
:1046000006C09FB7F8948C91832B8C939FBFDF914A
:10461000CF910895482F50E0CA018552994FFC016F
:104620002491CA018953994FFC0194914D54594FDB
:10463000FA013491332309F440C0222351F123308D
:1046400071F0243028F42130A1F0223011F514C08B
:104650002630B1F02730C1F02430D9F404C0809165
:1046600080008F7703C0809180008F7D80938000D1
:1046700010C084B58F7702C084B58F7D84BD09C01A
:104680008091B0008F7703C08091B0008F7D8093C0
:10469000B000E32FF0E0EE0FFF1FE156F94FA591B8
:1046A000B4912FB7F894662321F48C9190958923C7
:1046B00002C08C91892B8C932FBF0895682F70E0D6
:1046C000CB018552994FFC012491CB018953994F1D
:1046D000FC0144916D54794FFB019491992319F495
:1046E00020E030E03CC0222351F1233071F024302F
:1046F00028F42130A1F0223011F514C02630B1F099
:104700002730C1F02430D9F404C0809180008F7725
:1047100003C0809180008F7D8093800010C084B59D
:104720008F7702C084B58F7D84BD09C08091B000B1
:104730008F7703C08091B0008F7D8093B000892F68
:1047400090E0880F991F8755994FFC01A591B4916E
:104750008C9120E030E0842311F021E030E0C901A9
:10476000089508951F920F920FB60F9211242F9360
:104770003F934F938F939F93EF93FF938091C0004C
:1047800082FD1DC04091C6002091870730918807A7
:104790002F5F3F4F2F7730708091890790918A0764
:1047A0002817390771F0E0918707F0918807E95FD2
:1047B000F84F4083309388072093870702C0809189
:1047C000C600FF91EF919F918F914F913F912F9153
:1047D0000F900FBE0F901F901895E0911B08F0915D
:1047E0001C08E058FF4F81919191208131818058C0
:1047F0009F4F821B930B60E870E00E94652A892B13
:1048000011F00E94B12308951F920F920FB60F92DC
:1048100011242F933F938F939F93EF93FF932091B6
:104820000B0830910C0880910D0890910E08281704
:10483000390731F48091C1008F7D8093C10014C08D
:10484000E0910D08F0910E08E557F84F2081809116
:104850000D0890910E0801968F77907090930E0836
:1048600080930D082093C600FF91EF919F918F9147
:104870003F912F910F900FBE0F901F901895AF9200
:10488000BF92DF92EF92FF920F931F93CF93DF932C
:10489000EC017A018B01DD24403081EE580780E085
:1048A000680780E0780711F0DD24D39491E0A92E09
:1048B000B12CEC89FD89DD2069F0C50108A002C09A
:1048C000880F991F0A94E2F7808360E079E08DE316
:1048D00090E005C0108260E874E88EE190E0A801E5
:1048E00097010E94782A2150304040405040569510
:1048F00047953795279580E12030380720F0DD2057
:1049000011F0DD24D6CFE889F9893083EA89FB8963
:10491000208319A2EE89FF89408121E030E0C9019E
:104920000C8C02C0880F991F0A94E2F7482B408331
:10493000EE89FF894081C9010D8C02C0880F991F43
:104940000A94E2F7482B4083EE89FF894081C90130
:104950000E8C02C0880F991F0A94E2F7482B4083FF
:10496000EE89FF8980810F8C02C0220F331F0A94C9
:10497000E2F7209528232083DF91CF911F910F919B
:10498000FF90EF90DF90BF90AF900895DC011C96F0
:10499000ED91FC911D97E058FF4F819191912081FD
:1049A000318180589F4F821B930B60E870E00E941A
:1049B000652A0895DC011C96ED91FC911D97E05845
:1049C000FF4F20813181E058F040DF01AE57BF4FEB
:1049D0008D919C9111972817390719F42FEF3FEF0C
:1049E00007C08D919C91E80FF91F8081282F30E03E
:1049F000C9010895DC011C96ED91FC911D97E058CA
:104A0000FF4F20813181E058F040DF01AE57BF4FAA
:104A10008D919C9111972817390719F42FEF3FEFCB
:104A200010C08D919C911197E80FF91F20818D91F5
:104A30009C91119701968F77907011969C938E930D
:104A400030E0C9010895DC0191968C9191978823FB
:104A500039F05496ED91FC915597808186FFF9CFFE
:104A600091961C920895CF93DF93EC01EE85FF851C
:104A7000E058FF4F20813181E058F0402F5F3F4FD9
:104A80002F773070DF01AE57BF4F8D919C911197FA
:104A900028173907D1F3E058FF4F80819181E05802
:104AA000F040E80FF91F6083EE85FF85E058FF4F67
:104AB00031832083EE89FF89208181E090E00F8C93
:104AC00002C0880F991F0A94E2F7282B208381E007
:104AD00089A3EC89FD8980818064808381E090E0F6
:104AE000DF91CF910895109212081092110888EE6C
:104AF00093E0A0E0B0E08093130890931408A09393
:104B00001508B09316088EE691E0909310088093F4
:104B10000F0887E097E090931C0880931B088BE8B0
:104B200097E090931E0880931D0885EC90E0909389
:104B3000200880931F0884EC90E0909322088093D3
:104B4000210880EC90E0909324088093230881EC66
:104B500090E0909326088093250882EC90E0909353
:104B600028088093270886EC90E090932A08809389
:104B7000290884E080932B0883E080932C0887E049
:104B800080932D0885E080932E0881E080932F0884
:104B900008950895CF93DF930E9490220E94C92523
:104BA0000E94191BCDEED3E20E9491172097E1F3EA
:104BB0000E94ED23F9CFCF92DF92EF92FF920F93F5
:104BC0001F93CF93DF937C016B018A01C0E0D0E09B
:104BD0000FC0D6016D916D01D701ED91FC9101904F
:104BE000F081E02DC7010995C80FD91F0150104071
:104BF0000115110571F7CE01DF91CF911F910F9132
:104C0000FF90EF90DF90CF900895CF93DF93EC016A
:104C10006115710519F420E030E00FC0DB010D9043
:104C20000020E9F71197A61BB70BE881F9810280F4
:104C3000F381E02DAD0109959C01C901DF91CF9170
:104C400008954F925F927F928F929F92AF92BF9200
:104C5000CF92DF92EF92FF920F931F93DF93CF9348
:104C6000CDB7DEB7A1970FB6F894DEBF0FBECDBFAC
:104C70002C01742ECB01223008F42AE019A231E273
:104C8000C32ED12CCC0EDD1E822E9924AA24BB2447
:104C9000672D752FA50194010E94782A79018A0158
:104CA000C801B701A50194010E94322A472D461B75
:104CB0000894C108D1084A3014F4405D01C0495C31
:104CC000F6014083E114F1040105110521F07E2C69
:104CD0005F2DC801DDCFC201B6010E940526A19655
:104CE0000FB6F894DEBF0FBECDBFCF91DF911F91FD
:104CF0000F91FF90EF90DF90CF90BF90AF909F907B
:104D00008F907F905F904F900895DC0121153105C1
:104D100041F4ED91FC910190F081E02D642F099513
:104D200008950E9421260895CF92DF92EF92FF927C
:104D30000F931F93CF93DF93EC016A017B01211541
:104D4000310541F4E881F9810190F081E02D642F73
:104D500009951FC02A303105D1F477FF17C0E881CB
:104D6000F9810190F081E02D6DE209958C014427D5
:104D70005527BA014C195D096E097F09CE012AE059
:104D80000E9421269801280F391F04C02AE00E94A2
:104D900021269C01C901DF91CF911F910F91FF90B6
:104DA000EF90DF90CF9008950E94052608957F929E
:104DB0008F929F92AF92BF92CF92DF92EF92FF922B
:104DC0000F931F93CF93DF934C017A018B01722EC7
:104DD000CB01BA01A80197010E942E2A882321F055
:104DE000C4016FE371E021C0C0E0D0E05701680169
:104DF000E894D7F8C601B5012FEF3FEF4FE75FE723
:104E00000E942E2A882351F4C601B5012FEF3FEFEF
:104E10004FE75FE70E942328181614F0C1E0D0E0A6
:104E2000219739F0C40163E471E00E940526EC018A
:104E300093C0C801B7012FEF3FEF4FE75FE40E9437
:104E4000C729181654F0C801B7012FEF3FEF4FE7FD
:104E50005FEC0E942328882324F4C40167E471E0F6
:104E6000E4CFC801B70120E030E040E050E00E940C
:104E7000232887FD03C0C0E0D0E00EC0D401ED912F
:104E8000FC910190F081E02DC4016DE20995EC01E7
:104E900017FB109517F9109520E030E040E05FE334
:104EA000DD240BC0CA01B90120E030E040E251E44A
:104EB0000E9427289B01AC01D394D71498F3C80112
:104EC000B7010E94BF275B016C010E9494287B01FF
:104ED0008C01C401B801A7012AE030E00E948526B8
:104EE000C80FD91F772039F0C4016BE471E00E942C
:104EF0000526C80FD91FC801B7010E94C0289B0111
:104F0000AC01C601B5010E94BE2724C020E030E0FC
:104F100040E251E40E94CB297B018C010E948F2842
:104F20005B016C01CC24B7FCC094DC2CC401B6013D
:104F3000A5012AE030E00E949426C80FD91FC601BF
:104F4000B5010E94C2289B01AC01C801B7010E94B3
:104F5000BE277A947720D1F6CE01DF91CF911F91B1
:104F60000F91FF90EF90DF90CF90BF90AF909F9008
:104F70008F907F9008950E94D72608955058BB27A0
:104F8000AA270ED0B3C1A4D130F0A9D120F031F4BA
:104F90009F3F11F41EF499C10EF4E095E7FB64C144
:104FA000E92FB5D180F3BA17620773078407950715
:104FB00018F071F49EF5E4C10EF4E0950B2EBA2FB3
:104FC000A02D0B01B90190010C01CA01A00111240F
:104FD000FF27591B99F0593F50F4503E68F11A16BB
:104FE000F040A22F232F342F4427585FF3CF46954C
:104FF00037952795A795F0405395C9F77EF41F166E
:10500000BA0B620B730B840BBAF09150A1F0FF0F37
:10501000BB1F661F771F881FC2F70EC0BA0F621F23
:10502000731F841F48F4879577956795B795F79513
:105030009E3F08F0B3CF9395880F08F09927EE0FA5
:10504000979587950895ECD008F481E008950CD0E9
:105050004DC145D140F03CD130F021F45F3F19F013
:1050600003C151118EC131C152D198F39923C9F3B3
:105070005523B1F3951B550BBB27AA27621773075E
:10508000840738F09F5F5F4F220F331F441FAA1F12
:10509000A9F333D00E2E3AF0E0E830D091505040D2
:1050A000E695001CCAF729D0FE2F27D0660F771F80
:1050B000881FBB1F261737074807AB07B0E809F062
:1050C000BB0B802DBF01FF2793585F4F2AF09E3FF7
:1050D000510568F0C9C055C15F3FECF3983EDCF361
:1050E000869577956795B795F7959F5FC9F7880F70
:1050F000911D9695879597F90895E1E0660F771FC2
:10510000881FBB1F621773078407BA0720F0621B52
:10511000730B840BBA0BEE1F88F7E095089504D04B
:105120006894B1112EC10895FAD088F09F5790F07D
:10513000B92F9927B751A0F0D1F0660F771F881FBC
:10514000991F1AF0BA95C9F712C0B13081F018D181
:10515000B1E0089515C1672F782F8827B85F39F01F
:10516000B93FCCF3869577956795B395D9F73EF41B
:1051700090958095709561957F4F8F4F9F4F0895C3
:10518000E89409C097FB3EF49095809570956195E1
:105190007F4F8F4F9F4F9923A9F0F92F96E9BB2797
:1051A0009395F695879577956795B795F111F8CF13
:1051B000FAF4BB0F11F460FF1BC06F5F7F4F8F4F7E
:1051C0009F4F16C0882311F096E911C0772321F074
:1051D0009EE8872F762F05C0662371F096E8862F0C
:1051E00070E060E02AF09A95660F771F881FDAF763
:1051F000880F9695879597F90895ABD080F09F37E3
:1052000040F491110EF0BDC060E070E080E89FEBCB
:10521000089526F41B16611D711D811D2BC045C00C
:10522000990F0008550FAA0BE0E8FEEF16161706B7
:10523000E807F907C0F012161306E407F50798F01F
:10524000621B730B840B950B39F40A2661F0232B38
:10525000242B252B21F408950A2609F4A140A695B4
:105260008FEF811D811D089597F99F6780E870E099
:1052700060E00895882371F4772321F09850872BFC
:10528000762F07C0662311F499270DC09051862B05
:1052900070E060E02AF09A95660F771F881FDAF7B2
:1052A000880F9695879597F908959F3F49F09150FB
:1052B00028F4869577956795B7959F5F80389F4FBF
:1052C000880F9695879597F908959FEF80EC08953C
:1052D00000240A94161617061806090608950024D5
:1052E0000A9412161306140605060895092E03944F
:1052F000000C11F4882352F0BB0F40F4BF2B11F4C3
:1053000060FF04C06F5F7F4F8F4F9F4F089557FD21
:105310009058440F551F59F05F3F71F04795880F23
:1053200097FB991F61F09F3F79F0879508951216BA
:1053300013061406551FF2CF4695F1DF08C0161666
:1053400017061806991FF1CF869571056105089417
:105350000895E5DFA0F0BEE7B91788F4BB279F38B2
:1053600060F41616B11D672F782F8827985FF7CF46
:10537000869577956795B11D93959639C8F30895ED
:10538000E894BB2766277727CB0197F9089548DF74
:1053900008F48FEF08950BD0A9CF9ADF28F09FDF94
:1053A00018F0952309F060CF90CF1124EACFAFDF3A
:1053B000A0F3959FD1F3950F50E0551F629FF00128
:1053C000729FBB27F00DB11D639FAA27F00DB11D81
:1053D000AA1F649F6627B00DA11D661F829F22270A
:1053E000B00DA11D621F739FB00DA11D621F839F91
:1053F000A00D611D221F749F3327A00D611D231F67
:10540000849F600D211D822F762F6A2F11249F57B4
:1054100050408AF0E1F088234AF0EE0FFF1FBB1FD7
:10542000661F771F881F91505040A9F79E3F510576
:1054300070F01ACFA6CF5F3FECF3983EDCF3869571
:1054400077956795B795F795E7959F5FC1F7FE2B21
:10545000880F911D9695879597F90895E1DE880B41
:10546000990B0895629FD001739FF001829FE00D18
:10547000F11D649FE00DF11D929FF00D839FF00DD3
:10548000749FF00D659FF00D9927729FB00DE11D7F
:10549000F91F639FB00DE11DF91FBD01CF0111245C
:1054A0000895AA1BBB1B51E107C0AA1FBB1FA6176B
:1054B000B70710F0A61BB70B881F991F5A95A9F7BD
:1054C00080959095BC01CD01089597FB092E072684
:1054D0000AD077FD04D0E5DF06D000201AF47095DD
:1054E00061957F4F0895F6F7909581959F4F0895A8
:1054F000A1E21A2EAA1BBB1BFD010DC0AA1FBB1FD8
:10550000EE1FFF1FA217B307E407F50720F0A21B49
:10551000B30BE40BF50B661F771F881F991F1A94B6
:1055200069F760957095809590959B01AC01BD01E0
:10553000CF010895EE0FFF1F0590F491E02D09941F
:04554000F894FFCF0D
:10554400596F757243616C6C20004D7943616C6CCA
:10555400202020003E004D487A004E54484D4547D7
:105564004120362E350020442D537461720020539F
:1055740050384E5448202620535039414351006E30
:10558400616E00696E66006F7666002E002C01FA6B
:10559400000100000000511C0D1C00000000EE1E64
:1055A400BD1E761E7F1E941EA51E0000000033251E
:0A55B400DB25C624FA24DA2423259F
:00000001FF
